:1000000061C087C070C285C084C084C082C081C006
:1000100080C07FC07EC07DC017C17BC07AC0010197
:10002000010102030406090E162338596A7F97B4AA
:10003000D6FF1400081400080E140004080E140063
:100040000305080E140004080B0E11140003050824
:100050000B0E1014000305080B0E101214000800FC
:100060000E00080E0004080E000305080E00040828
:100070000E1100080E1100F3F404080E1012140003
:10008000080A0C0E0F10121400080EED14000405DF
:10009000060700041400040E1400040810140004E1
:1000A000080F1114000305080A0E0004080B0E00C7
:1000B000EEEDECEB140E08040004080E00EBECED82
:1000C000EEF3F41411241FBECFE5D1E0DEBFCDBFA7
:1000D00020E0A0E6B0E001C01D92AA37B207E1F728
:1000E000EBE7F0E085E5808781E08383148212826C
:1000F000868311828BE0818788E58287E1E6F0E0E4
:100100008DEF87838EEF8583712C55245A949DD073
:1001100012C276CF189525B7277E25BF29B7226052
:1001200029BF21E022BF019728F020E188952150C6
:10013000E9F7F9CF089588EE93E0EDCF369A369936
:10014000FECF95B18091600089270895CF93C72D88
:1001500081E0870D8F73782E662D90E0DED16FEFF2
:100160008C2F90E0CF91D9C1FF920F931F93CF9323
:10017000DF93F82E0CE710E0CEE7D0E0F11005C0D9
:10018000CE01C3D1F801808304C0F8016081CE01A3
:10019000C4D121970F5F1F4FC437D10579F7DF9185
:1001A000CF911F910F91FF900895D0DF81E0DCCFB8
:1001B000EF92FF920F931F93CF93C82F8B0182E290
:1001C000E82E80E0F82ECC2361F0F70184918BBDFE
:1001D000C801A1DF1BBCC8019EDFC8019CDFC15064
:1001E000F2CFCF911F910F91FF90EF900895CF9391
:1001F000DF93D82F64E170E08AE0DADF84EF91E0EA
:100200008ADF8D2F64E675D1CAE06C2F72D1892FF9
:1002100068EC70E0CDDF8FDF8D2F6C2F6AD1D92F86
:1002200068D1892F68EC70E0C3DF85DF68EC70E08F
:100230008D2FBEDF80DF64E170E08AE0B9DF84EFFC
:1002400091E0DF91CF9167CF189510927A0087E700
:1002500090E05BD1853519F0612CA7DF11C0712CBE
:10026000872D90E052D1682E8F3F19F080E07CDF1F
:1002700007C0872D91E0970D792E803488F3F6CF53
:1002800090918400D0917E0010917F00C0917C00FD
:10029000CC2319F010E0D0E09AE19F5F80E040E0CD
:1002A00050E062E370E0992379F09B012F5F3F4FAC
:1002B000F9013197E491EE2319F0822F861BF6CFD6
:1002C0009150AB01B901EFCF982F6D2F70E0A82F9F
:1002D000B0E0E92FF0E0112321F09D012E1B3F0B30
:1002E00005C09F0121503109260F371F3197E40FB8
:1002F000F51F049126593F4FF9010083915049F7AA
:100300008D0F80938600DD2371F0112329F0282FB3
:1003100030E02150310902C020E030E0F901E65917
:10032000FF4F91E0908397E0980F292F2150E22F03
:10033000E81BF0E0E354FF4FE491A22FB0E0A65990
:10034000BF4FEC932813F2CFE92FF0E0E759FF4FAE
:1003500021E040916A003081431320E0921B90938A
:100360008700262D253FE8F5352D3D30B0F49091DE
:1003700088009F3F29F480917A008093880006C00E
:1003800091E0960D692E981708F0612C80918800F5
:100390008F5F8F718093880024C020917A00209312
:1003A00088003132C0F420918100222311F0CC2347
:1003B00039F091E0960D692E981798F0612C11C0D4
:1003C000262D6816D9F3662019F02150622E09C037
:1003D0009150692E06C0C111F1CF80917D00882314
:1003E00069F3512C8FEF8DBD80E68CBDAB9A8FE306
:1003F00084BB8FE187BB8CEE88BB81E083BF8ABD65
:1004000080BF8BB780628BBF8AB785608ABF85B794
:10041000806285BF78948CE287B986EC86B936997C
:10042000FECF8FEF809360008CE291E074DE86DE79
:10043000DEDEFACF112416B81BBC87B38C7E87BBD7
:10044000C29820E061E031E040E050E0E8E0999BB4
:1004500006C0CA010197F1F78AB785608ABF86B3E3
:100460008E27999B03C0511003C035C0811107C06E
:1004700090E2951590F5211130C060E039E0952D9E
:1004800071E0923208F070E0970F592E913209F422
:10049000C29A611106C0211103C0882311F0C298CD
:1004A00021E0999885B7877E806185BFA895832FC5
:1004B000887011F480E401C080E6816081BD85B759
:1004C000846885BF8B7F85BF78948895F89481B5C3
:1004D0008F7B81BDBCCF8111D2CF8FE58DBF81E0F5
:1004E0008EBF1FBEB2DE999A552011F0189501C03B
:1004F000A1DF991B79E004C0991F961708F0961B9D
:10050000881F7A95C9F780950895E199FECF1FBAA3
:100510008EBBE09A99278DB30895262FE199FECFDF
:100520001CBA1FBA8EBB2DBB0FB6F894E29AE19AA3
:0A0530000FBE01960895F894FFCF66
:00000001FF
